:020000040800F2
:1000000000070020F1010008B1240008692400085D
:10001000912400086924000889240008F3010008DD
:10002000F3010008F3010008F30100084D35000852
:10003000F3010008F3010008F3010008F3010008D0
:10004000F3010008F3010008F3010008F3010008C0
:10005000F3010008F3010008154300083D430008C0
:10006000654300088D430008B5430008F30100080C
:10007000F3010008F3010008F3010008F301000890
:10008000F3010008F3010008F30100081D24000833
:100090004924000859240008F3010008DD43000842
:1000A000F3010008F3010008F3010008F301000860
:1000B000C5440008F3010008F3010008F30100083B
:1000C000F3010008F3010008F3010008F301000840
:1000D000F3010008F3010008B1440008F30100082F
:1000E00041440008F3010008F3010008F30100088F
:1000F000F3010008F3010008F3010008F301000810
:10010000F3010008F3010008F3010008F3010008FF
:10011000F3010008F3010008F3010008F3010008EF
:10012000F3010008F3010008F3010008F3010008DF
:10013000F3010008F3010008F3010008F3010008CF
:10014000F3010008F3010008F3010008F3010008BF
:10015000F3010008F3010008F3010008F3010008AF
:10016000F3010008F3010008F3010008F30100089F
:10017000F3010008F3010008F3010008F30100088F
:10018000F3010008F3010008F3010008F30100087F
:10019000F3010008F3010008F3010008F30100086F
:1001A000F3010008F3010008F3010008F30100085F
:1001B000F3010008F3010008F3010008F30100084F
:1001C000F3010008F3010008F3010008F30100083F
:1001D000F3010008F3010008F3010008F30100082F
:1001E000C10F000800000000000000000000000037
:1001F00002E000F000F8FEE772B6374880F30888A6
:10020000364880F3098836483649086040F20000D5
:10021000CCF200004EF63471CEF200010860BFF35C
:100220004F8FBFF36F8F40F20000C0F2F0004EF628
:100230008851CEF200010860BFF34F8FBFF36F8F7C
:100240004FF00000E1EE100A4EF63C71CEF20001D4
:100250000860062080F31488BFF36F8F03F064FEFC
:1002600003F0F6FE4FF055301F491B4A91423CBF48
:1002700041F8040BFAE71D49184A91423CBF41F886
:10028000040BFAE71A491B4A1B4B9A423EBF51F82E
:10029000040B42F8040BF8E700201849184A914271
:1002A0003CBF41F8040BFAE703F042FE03F01EFFE7
:1002B000144C154DAC4203DA54F8041B8847F9E797
:1002C00000F042F8114C124DAC4203DA54F8041B12
:1002D0008847F9E703F02ABE00070020002300202A
:1002E0000000000808ED00E00001002000070020E9
:1002F000E04C000800230020802300208023002001
:10030000C44F0020E0010008E4010008E4010008F7
:10031000E40100082DE9F04F2DED108AC1F80CD052
:10032000C3689D46BDEC108ABDE8F08F002383F3BF
:1003300011882846A047002003F064FAFEE703F086
:10034000EDF900DFFEE70000F8B500F04BFE03F02A
:1003500085FD074603F0D4FD064600283DD12B4B12
:100360009F423AD001339F423AD0294B27F0FF02F7
:100370009A4238D1F8B200F03FFC354642F2107490
:1003800000F040FC08B10024254601F055F970B397
:10039000032000F043F80024254636B11D4B9F4250
:1003A00003D003F0A5FD00242546002003F060FDE6
:1003B000194B1B691B041FD40DB100F045F800F068
:1003C0008FFC02F07DF80546C4B102F079F8401BBD
:1003D000A04213D900F038F8F3E735460024CFE700
:1003E00004460125CCE705464FF47A74C8E7B4F516
:1003F0007A7F08BF0125D0E70024E0E700F0B8FCD1
:100400004FF47A7003F004FADEE700BF010007B092
:10041000000008B0263A09B000040240084B1870EA
:1004200003280CD8DFE800F008050208022000F0DD
:1004300037BE022000F02ABE024B00225A607047ED
:10044000802300208423002010B501F0F5F830B19E
:10045000204B03221A70204B00225A6010BD1F4B04
:100460001F4A1C4619680131F8D004339342F9D170
:1004700062681C4B9A42F1D91B4B9B6803F10063E5
:1004800003F580339A42E9D203F006FD03F018FD2C
:10049000002000F0C1FD0220FFF7C0FF134B1A6CD3
:1004A00000221A64196E1A66196E596C5A64596ED4
:1004B0005A665B6E72B64FF0E0233021C3F8084DE8
:1004C000D4E9003281F311889D4683F308881047F0
:1004D000C4E700BF8023002084230020000001081F
:1004E00020000108FFFF0008002300200038024020
:1004F000094A136849F2690099B21B0C00FB0133E9
:100500001360064B186844F2506182B2000C01FB84
:100510000200186080B270471823002014230020C6
:1005200010B500211022044600F0D6FD034B03CB8A
:10053000206061601868A06010BD00BF107AFF1FC6
:10054000F0B5ADF54F7D6CAC4FF4C47207460D4667
:100550002046002100F0C0FD01F0B2FF264B4FF411
:100560007A72B0FBF2F0186093E80700022384E887
:1005700007000DF5E9702382FFF7D2FF4FF4A24385
:100580001E49238407A804F0B3FA152384F83231F6
:100590000DF2E32207AB0DF12C0C1E4603CE66458F
:1005A00010605160334602F10802F6D130681060E5
:1005B000337913710DAE31460122204600F0D8FD8B
:1005C00000230393AB7E029305F11903019380B2DC
:1005D0000123CDE904600093E97E05A3D3E900235C
:1005E000384602F083FB0DF54F7DF0BDAFF3008080
:1005F0009E6AC421818A46EE8C230020004B0008AD
:100600002DE9F0412C4C237ADAB080460D465BBBD5
:1006100027A9284600F0D2FE0746002842D19DF8BF
:100620009D60C82E3ED801464FF4A662204600F0D9
:1006300053FD4FF48073C4F8F8314FF40073C4F8DD
:100640000C334FF44073C4F8203432460DF19E0150
:1006500004F1090000F02EFD26449DF89C307772CD
:1006600023720BB9EB7E23728122002106AC27A8EE
:1006700000F032FD0122214627A800F0E5FE00230C
:100680000393AB7E029305F1190380B201932823F3
:10069000CDE904400093E97E05A3D3E90023404659
:1006A00002F024FB5AB0BDE8F08100BFAFF3008038
:1006B00026417272DF25D7B7D4330020F0B5254E1E
:1006C0004FF48A7505FB0065F1B096F8D83085F8CF
:1006D000DC300024D822214685F8E8403AA800F012
:1006E000FBFC06F1090000F0EFFCD5F8E4308DF8D2
:1006F000F000C2B206AF06F109010DF1F100CDE93B
:100700003A3400F0D7FC394601223AA800F0D2FE74
:1007100080B2CDE9047008230127CDE9023706F144
:10072000D803019330230093317A0B4807A3D3E910
:10073000002302F0DBFAA04206DD01F0C1FEC5F89D
:10074000E000384671B0F0BD2046FBE778F6339FF5
:1007500093CACD8DD4330020A43300202DE9F0417D
:100760001D4D1E4E1E4F86B0284602F0EBFA034682
:1007700058B30024CDE90344ADF81440027B8DF852
:10078000142099684068029403AA03C21B68DFF82A
:10079000548043F00043029301F094FE821941F12A
:1007A0000003009402A9384601F028F9A04205DDB3
:1007B000284602F0CBFA88F80040D5E798F80030D8
:1007C000072B05D8013388F8003006B0BDE8F0816A
:1007D000014802F0BBFAF8E7A433002040420F00C2
:1007E000103900200939002070B50D4614461E4608
:1007F00002F0D8F950B9022E10D1012C0ED112A35B
:10080000D3E90023C5E90023012007E0282C10D0FC
:1008100005D8012C09D0052C0FD0002070BD302C3C
:10082000FBD10BA3D3E90023ECE70BA3D3E900230F
:10083000E8E70BA3D3E90023E4E70BA3D3E9002304
:10084000E0E700BFAFF30080401DA12026812A0B06
:1008500078F6339F93CACD8D9E6AC421818A46EE75
:1008600026417272DF25D7B7F017304A39059E56F8
:1008700038B505460E4C0021013500F0EFFBA4F819
:100880002C55B4F82C0500F0D1FB78B1B4F82C0548
:1008900000F0DCFB014648B9B4F82C0500F0DEFBA3
:1008A000B4F82C350133A4F82C35EAE738BD00BF85
:1008B000D433002010B50A4B0A4A1A6003F580535E
:1008C00093F870203AB9DC6E2CB1204600F02CFF72
:1008D000204601F069F8BDE81040034800F024BF4D
:1008E00010390020544B0008684900202DE9F04FD2
:1008F0008FB000AF05460C4602F054F900284BD1EA
:10090000237E022B1BD1E38A012B18D101F0D8FDE5
:100910000646FFF7EDFD03464FF4C870DFF8D482BA
:10092000B3FBF0F206F5167602FB103316FA83F3EA
:10093000C8F80030E37E33B9A74B00221A703C3769
:10094000BD46BDE8F08F07F12401204600F0EAFC27
:100950000028F4D107F11400FFF7E2FD97F82640D4
:1009600007F11401224607F1270004F08FF8002850
:10097000E2D10F2C08D8984B1C70D8F80030A3F5A2
:100980001673C8F80030DAE797F824100029D6D09B
:10099000284602F0FFF8D2E7E38A282B33D010D89C
:1009A000012B2BD0052BCAD1BFF34F8F8B498C4B1A
:1009B000CA6802F4E0621343CB60BFF34F8F00BFFD
:1009C000FDE7302BBBD1874EE17E327A9142B6D122
:1009D000607E3146002291F8DC50854200F0AD8007
:1009E0000132042A01F58A71F5D1326840F6B83136
:1009F000FA328A4294BF32603160A0E7214628462D
:100A0000FFF79EFD9BE721462846FFF7F9FD96E795
:100A1000B2F8EC507B6005F103094FEA99094FEAFF
:100A20008902D11DC908A8EBC1039D46EB460021F0
:100A3000584600F051FB04F1EE012A463144584675
:100A400000F038FB7B6813B9012000F0E5FA96F856
:100A5000D20000F0EBFA044630B9307200F006FB29
:100A6000204600F0D9FAB0E0D6F8D4203AB996F88A
:100A7000D200B6F82C25824201D8FFF7F9FED6F84D
:100A8000D4202A44944208D296F8D200B6F82C25F5
:100A90000130824201D8FFF7EBFE70685FFA89F2FD
:100AA000594600F021FB08B9C54679E0726896F80E
:100AB000D2002A447260D6F8D42005EB0209C6F8A9
:100AC000D49000F0B3FA814509D396F8D220D6F835
:100AD000D4000132001B86F8D220C6F8D400FF2DC6
:100AE0000FD80024347200F0C1FA204600F094FAC6
:100AF00000F0A2FD3C4B188108B9FFF7A5FCC546E4
:100B00001DE7BB6896F8D9000AFB0362FB68D2F8C0
:100B1000E41082F8E83001F58061C2F8E030C2F8F4
:100B2000E410FFF7CBFDFFF719FE96F8D92001324C
:100B300002F0030286F8D920B6E74FF48A7A0AFB5E
:100B400002F505F1EA013144204600F0E7FCF860C7
:100B500000287FF4F4AE3544012285F8E82001F046
:100B6000AFFCD5F8E020D6ED007ADFED206A801AE0
:100B7000192838BF192040F6B832904228BF1046D5
:100B8000B8EE677A07EE900AF8EEE77A67EEA67A93
:100B9000DFED176AE7EE267AFCEEE77AC6ED007A1B
:100BA00096F8D9307168BB600AFB03F4321992F8E9
:100BB000E8505DB1D2F8E4308B42E8463FF428AF0C
:100BC000002182F8E810C2F8E010C5467368064AB2
:100BD0009B0A01331381B2E69D33002000ED00E053
:100BE0000400FA05D43300208C230020CDCCCC3D6A
:100BF0006666663FA0330020014B1870704700BF47
:100C00009823002030B54FF000542C4B22689A42B4
:100C100085B023D1637D0BB3294A2A481370237D05
:100C200003724FF48073C0F8F8314FF40073C0F8CA
:100C30000C3300254FF44073C0F820342249C0F82B
:100C4000E450C922093000F035FA2046E022294656
:100C500000F042FA0124204605B030BD03F05AF9F5
:100C6000044608B90024F6E7184A194D136C43F0FE
:100C700000731364AA6D174B9A42F3D12B6E013B9C
:100C80007E2BEFD8144A07CA01AB83E80700184649
:100C9000032100F09FFC6B6D83424FF00003E1D114
:100CA0002A6D8A4201BFAB65054B2A6E1A7003BFDD
:100CB0000A4BEA6D1A601C46CDE700BF9AAD44C5E9
:100CC00098230020D4330020160000200038024072
:100CD000006600405041A0B058660040102300203C
:100CE00037B51A4D00F0A8FC02236B71184B288110
:100CF00019681848012201F07DFA00230193164B70
:100D0000164900931648174B4FF4805201F01AFF12
:100D1000154B197811B1124801F03CFF01F0D0FBDE
:100D20000446FFF7E5FB4FF4C873B0FBF3F202FB98
:100D3000130304F5167010FA83F00C4B186003F0DF
:100D4000DFF808B10F232B8103B030BD8C230020C6
:100D50001023002010390020E90700089C23002000
:100D6000A4330020ED08000898230020A0330020C1
:100D70002DE9F04F2DED028B0FF23829D9E90089CA
:100D8000834C93B00BAE9FED7E8BFFF7E7FC814F5A
:100D9000DFF828A200230A93ADF834300B93736078
:100DA0004FF0000B5B468DED008B01250DF11D0210
:100DB00007A938468DF81C508DF81DB001F0C8F910
:100DC0009DF81C30002B40F0A580204601F0EAFE83
:100DD0000646002845D1704F01F072FB3B689842EF
:100DE0003FD301F06DFB8246FFF782FB4FF4C873DF
:100DF000B0FBF3F202FB13030AF5167010FA83F04E
:100E00003860664F97F800B0CBF1100ABBF1000FC5
:100E100014BF33462B465FFA8AFA0EA88DF82830A5
:100E2000FFF77EFBBAF1060F28BF4FF0060A0EABA4
:100E300003EB0B0152460DF1290000F03BF90AAB20
:100E40000393182302930AF10102554BD2B2CDE964
:100E50000053049220464CA3D3E9002301F0E8FE9E
:100E60003E7001F02DFB4F4A4F4D1368C31AB3F586
:100E70007A7F2ED3106001F025FB02460B462046F8
:100E800001F06EFF204601F08DFE10B32B7A474E25
:100E9000002B14BF03230223737101F011FB0EAF6B
:100EA0004FF47A730122B0FBF3F0394630603046DC
:100EB00000F010FA182302933D4B019380B240F2E8
:100EC0005513CDE90370009342464B46204601F08E
:100ED000AFFE2B7A93B101F0F3FA002607464FF4E8
:100EE0008A7A95F8D900304400F003000AFB0053D9
:100EF00093F8E82092B30136042EF2D1C82002F014
:100F000087FC2B7A002B7FF43DAF13B0BDEC028B36
:100F1000BDE8F08FDAF8143083F48063CAF8143037
:100F2000594610220EA800F0D7F80DF11E0308AAAA
:100F30000AA9384600F068FE96E803000FAB83E884
:100F400003009DF834308DF844300A9B0E930EA9AF
:100F5000DDE90823204602F0D7F821E7D3F8E020A6
:100F600042B12B68FA2B38BFFA23BA1A0533B2EB19
:100F7000430FC0D3FFF7A2FB0028BCD1BEE700BFE0
:100F80000000000000000000401DA12026812A0B67
:100F9000A433002010390020A03300209D3300200E
:100FA0009C33002004390020D43300208C230020FF
:100FB00008390020F1C6A7C1D068080F0000024020
:100FC00008B5054800F0BEFEBDE80840034A0449E4
:100FD000002003F037BD00BF10390020304A002048
:100FE000B508000870B502F0E7FD094E094D3080E4
:100FF000002428683388834208D902F0D7FD2B6883
:1010000004440133B4F5803F2B60F2D370BD00BFC0
:10101000244A0020F849002002F07EBE00F1006062
:10102000920000F5803002F00DBE0000054B1A68FA
:10103000054B1B889B1A834202D9104402F0B6BDAF
:1010400000207047F8490020244A0020024B1B680A
:10105000184402F0B3BD00BFF8490020024B1B68E2
:10106000184402F0C3BD00BFF8490020064991F8BA
:10107000243033B10023086A81F824300822FFF7B6
:10108000CDBF0120704700BFFC490020022802BFED
:10109000024B4FF080629A61704700BF000002402F
:1010A000022802BF024B4FF480629A61704700BF72
:1010B0000000024010B50023934203D0CC5CC4541E
:1010C0000133F9E710BD000003460246D01A12F9B9
:1010D000011B0029FAD1704702440346934202D013
:1010E00003F8011BFAE770472DE9F8431F4D14463A
:1010F00095F824200746884652BBDFF870909CB3D1
:1011000095F824302BB92022FF2148462F62FFF7A3
:10111000E3FF95F82400C0F10802A24228BF22464E
:10112000D6B24146920005EB8000FFF7C3FF95F869
:101130002430A41B1E44F6B2082E17449044E4B297
:1011400085F82460DBD1FFF791FF0028D7D108E0B4
:101150002B6A03EB82038342CFD0FFF787FF00287F
:10116000CBD10020BDE8F8830120FBE7FC4900203B
:101170002DE9F3470D46044600219046284640F2EB
:101180007912FFF7A9FF234620220021284601F00B
:101190005DFF231D02222021284601F057FF631D19
:1011A00003222221284601F051FFA31D03222521FD
:1011B000284601F04BFF04F108031022282128469D
:1011C00001F044FF04F1100308223821284601F001
:1011D0003DFF04F1110308224021284601F036FFAB
:1011E00004F1120308224821284601F02FFF04F1E0
:1011F000140320225021284601F028FF04F118038F
:1012000040227021284601F021FF04F1200308222A
:10121000B021284601F01AFF04F121030822B82169
:10122000284601F013FF04F12207C0263B46314651
:1012300008222846083601F009FFB6F5A07F07F11D
:101240000107F3D194F832308DF8073031460DF1B3
:1012500007030822284601F0F9FE002604F1330AAC
:101260009DF807304FEAC6099E4209F5A47720D3BE
:1012700094F83231502B28BF50238DF80730B8F145
:10128000000F08D139460DF107030722284601F067
:10129000DDFE09F24F17002604F233149DF80730E3
:1012A0009E4207EBC6010DD30731C80802B0BDE866
:1012B000F0870AEB060308223946284601F0C6FEED
:1012C0000136CDE7A3190822284601F0BFFE0136FA
:1012D000E4E7000013B504460846002101602346F8
:1012E000C0F803102022019001F0B0FE0198231DE8
:1012F0000222202101F0AAFE0198631D032222216F
:1013000001F0A4FE0198A31D0322252101F09EFEF9
:10131000019804F108031022282101F097FE07200C
:1013200002B010BDF7B5047F05460E462CB1838A86
:10133000122B02D9012003B0F0BD00231946072269
:101340000096284601F046FD731C009301220023FD
:101350000721284601F03EFDD4B9B31C00930522B5
:1013600023460821284601F035FD0D24B378102BC3
:10137000E0D83746B278BB1B934210D32B7FA88AA4
:101380000734E408B3B9844294BF00200120D2E7B7
:10139000AB8ADB00083BDB08B3700824E6E7FB1CE4
:1013A0000093214600230822284601F013FD08344B
:1013B0000137DFE7201A18BF0120BCE7F7B5047F2B
:1013C00005460E462CB1838ACA2B02D9012003B0F0
:1013D000F0BD0023194600960822284601F0FAFCC9
:1013E000731CD4B90822009311462346284601F005
:1013F000F1FC10247378C82BE8D8012372785F1CA5
:10140000013B934210D32B7FA88A0734E408B3B979
:10141000844294BF00200120D9E7AB8ADB00083B5F
:10142000DB0873700824E5E7F319009321460023D5
:101430000822284601F0CEFC08343B46DEE7201A9D
:1014400018BF0120C3E70000F7B50D460446002190
:10145000164628468122FFF73FFE23460822002138
:10146000284601F0F3FD94F901206378002AB8BF03
:101470007F238DF807309EB90DF10703072208215D
:10148000284601F0E3FD0F27002602349DF80730BF
:101490009E4207EBC60105D30731C80803B0F0BD73
:1014A0000827F1E7A3190822284601F0CFFD0136ED
:1014B000ECE70000F7B50E4605460021144630461D
:1014C000CE22FFF709FE2B4628220021304601F0EC
:1014D000BDFD2B7AC82B28BFC8238DF807308CB9E7
:1014E0000DF1070308222821304601F0AFFD30241A
:1014F0002F469DF807207B1B934205D3E01DC008B3
:1015000003B0F0BD2824F3E707F1090321460822C0
:10151000304601F09BFD08340137EAE7F7B5047F58
:1015200005460E4634B1838AB3F5827F02D9012085
:1015300003B0F0BD0096012310220021284601F0DF
:1015400049FCDCB9B31C009309222346102128462C
:1015500001F040FC19247388B3F5807FE7D8374643
:101560007288BB1B934210D32B7FA88A0734E408F0
:10157000B3B9844294BF00200120D9E7AB8ADB00D5
:10158000103BDB0873801024E5E73B1D00932146E8
:1015900000230822284601F01DFC08340137DFE74C
:1015A000201A18BF0120C3E730B5094D0A44914203
:1015B0000DD011F8013B5840082340F30004013BD3
:1015C0002C4013F0FF0384EA5000F6D1EFE730BD62
:1015D0002083B8EDF7B54FF0FF33DFF854C0DFF8E4
:1015E00054E000EB81011A4688421CD050F8044BAD
:1015F000019401AF042417F8015B82EA0562082513
:10160000DB18164605F1FF355241002EBCBF83EAB8
:101610000C0382EA0E0215F0FF05F1D1013C14F033
:10162000FF04E8D1E0E7D843D14303B0F0BD00BFE9
:101630009336EAA9EBE1F042F7B5354A10685168F4
:101640006B4603C36A4633493348082303F02EFA36
:10165000044688BB0A25314A106851686B4603C3AB
:101660006A462F492C48082303F020FA0446002834
:1016700045D00369B3F5E02F41D8B0F86620512A70
:101680003DD1284A024402F15C018B4237D35C3BD6
:10169000214900209E1AFFF787FF3246074604F1D2
:1016A00064010020FFF780FFA3689F4227D1E36811
:1016B000984208BF002522E00369B3F5E02F25D842
:1016C000428B512A20D1174A024402F110018B4269
:1016D00018D3103B104900209D1AFFF765FF2A46DA
:1016E000064604F118010020FFF75EFFA3689E4242
:1016F00002D1E368984201D00D25ACE700252846C9
:1017000003B0F0BD1025A6E70C25A4E70B25A2E742
:10171000184B0008DCFF060000000108214B000800
:1017200090FF06000800FFF710B5037C044613B9CC
:10173000006803F0A3F9204610BD00000023BFF3AA
:101740005B8FC360BFF35B8FBFF35B8F8360BFF3BF
:101750005B8F7047BFF35B8F0068BFF35B8F704791
:1017600070B505460C30FFF7F5FF05F10806044695
:101770003046FFF7EFFFA04206D930466D68FFF70D
:10178000E9FF2544281A70BD3046FFF7E3FF201A11
:10179000F9E7000070B50546406898B105F108000A
:1017A000FFF7D8FF05F10C0604463046FFF7D2FFDD
:1017B0008442304694BF6D680025FFF7CBFF013CA3
:1017C0002C44201A70BD000038B50C460546FFF7C2
:1017D000C7FFA04210D305F10800FFF7BBFF044488
:1017E0006868B4FBF0F100FB1144BFF35B8F01208C
:1017F000AC60BFF35B8F38BD0020FCE72DE9F04102
:10180000144607460D46FFF7C5FF844228BF04462D
:10181000D4B1B84658F80C6B4046FFF79BFF3044F4
:10182000286040467E68FFF795FF331A9C4203D834
:101830006C600120BDE8F0816B60A41B3B68AB606D
:101840002044E8600220F5E72046F3E738B50C466F
:101850000546FFF79FFFA04210D305F10C00FFF7EC
:1018600079FF04446868B4FBF0F100FB1144BFF356
:101870005B8F0120EC60BFF35B8F38BD0020FCE77D
:101880002DE9FF41884669460746FFF7B7FF6C46DA
:1018900006B204EBC6060025B44209D0626820688F
:1018A00008EB0501FFF706FC636808341D44F3E705
:1018B00029463846FFF7CAFF284604B0BDE8F08144
:1018C000F8B505460C300F46FFF744FF05F1080652
:1018D00004463046FFF73EFFA042304688BF6C68A2
:1018E000FFF738FF201A386020B130462C68FFF728
:1018F00031FF2044F8BD000073B5144606460D467E
:10190000FFF72EFF844228BF04460190DCB101A9F5
:101910003046FFF7D5FF019B33B93268C5E9023382
:10192000C5E9002401200CE09C4238BF01942860E6
:10193000019868608442F5D93368AB60241AEC6082
:10194000022002B070BD2046FBE700002DE9FF41F8
:101950000F466946FFF7D0FF6C4600B204EBC005A6
:101960000026AC4209D0D4F8048054F8081BB819FA
:101970004246FFF79FFB4644F3E7304604B0BDE81C
:10198000F081000038B50546FFF7E0FF0446014648
:101990002846FFF719FF204638BD00000121884284
:1019A00038BF084603F054B808B103F067B8704771
:1019B00010B4026854681A4623465DF8044B184771
:1019C00000207047002070477047000000207047DB
:1019D0000E20704700F5805090F8D800C0F340000A
:1019E0007047000000F5805090F9E000704700005B
:1019F00000F58050C0F8DC1001207047F7B50C6886
:101A0000BDF8207014F0005473D10D7B082D70D8F0
:101A1000302585F31188456AAE6876010CD4AC6830
:101A2000240108D4AC6814F0805460D184F3118888
:101A3000204603B0F0BD01240E6804F1180C002EFE
:101A4000B8BFF6004FEA0C1CB4BF46F0040676059A
:101A500045F80C600E680FFA84FC16F0804F18BF32
:101A600005EB0C1E05EB0C1C1EBFDEF8806146F07A
:101A70000206CEF880610E7BCCF8846105EB04157C
:101A80008E68C5F88C614E68C5F88861DCF88051B5
:101A900045F00105CCF8805141F2780500EB441C7B
:101AA000660105EB4414AC440444CCE900230D4624
:101AB000083401F10C0C55F804EB44F804EB6545CF
:101AC000F9D12D882580841904F5805407F0030589
:101AD00094F8946026F00B06354384F89450002463
:101AE00084F31188009700F035FD0120A1E702245E
:101AF000A2E74FF0FF309CE713B500F58054019149
:101B0000E06EFFF747FE1F280AD90199E06E2022F8
:101B1000FFF7B6FEA0F120035842584102B010BDB5
:101B20000020FBE708B5302383F3118800F58050CF
:101B3000C06EFFF703FE002383F3118808BD000089
:101B400000220260828142608260704710B50022EC
:101B50000023C0E900230023044603810C30FFF773
:101B6000EFFF204610BD0000F0B5054600F580509F
:101B70000C4690F8D83013F0040FC3F3800108BF6F
:101B8000114661F3820380F8D83005EB441303F566
:101B90008453103389B01B79D8074FEA44162FD5E8
:101BA00082B319072ED46846FFF7D0FF05EB441324
:101BB00003F5845303AA03F108071868596814460B
:101BC00003C40833BB422246F7D1186820609B88C3
:101BD000A380DDE90E23CDE900230123ADF8083011
:101BE0002B6869461B6C28469847354405F5845593
:101BF00010352B791A075CBF43F008032B7101E005
:101C0000002AF2D109B0F0BD2DE9F0479A4688B01C
:101C1000074688469146302383F3118807F58054A0
:101C20006846FFF793FFE06EFFF79AFD1F282AD959
:101C3000E06E20226946FFF7A5FE202823D103ADE0
:101C4000444605AB2E4603CE9E4220606160354679
:101C500004F10804F6D130682060B388A380DDE980
:101C60000023C9E90023BDF80830AAF8003000239A
:101C700083F3118853464A464146384608B0BDE8CA
:101C8000F04700F02BBC002080F3118808B0BDE8BD
:101C9000F08700002DE9F84F182204460F46043063
:101CA0000021FFF719FA2046234B40F8283BFFF7A5
:101CB00047FF04F13800FFF749FF04F1580804F525
:101CC00082554646183530462036FFF73FFFAE4274
:101CD000F9D104F580554FF480534FF00009C5E960
:101CE0001739C5F858800123EE6604F5875804F5C6
:101CF0008456C5F8649085F8683085F870301836D9
:101D000008F118084FF0000A4FF0000B46E908AB45
:101D1000A6F11800FFF714FF203646F8289C464528
:101D2000F4D185F8E07017B1044800F0C3FB044B10
:101D300063622046BDE8F88F544B00082C4B000826
:101D40000064004010B5044B197804464A1C1A7010
:101D5000FFF7A0FF204610BD2C4A00202DE9F047D8
:101D6000002950D0294B2A4FB7FBF1F599428CBF7F
:101D70000A231123581EB5FBF3FC03FB1C53C4B20A
:101D80002BB102280346F5D80020BDE8F0870CF1FE
:101D9000FF36B6F5806FF7D2C4EBC40E0EF1030325
:101DA0004FEAE309C3F3C703A4EB030809F1010AEF
:101DB0004FF47A755FFA88F009FB05555AFA88F8EE
:101DC000B5FBF8F5B5F5617FC1BF0EF1FF33C3F385
:101DD000C703E01AC0B25C1C50FA84F40CFB04F494
:101DE000B7FBF4F4A142CFD1013BDBB20F2BCBD830
:101DF0000138C0B20728C7D8002110711680917031
:101E0000D3700120C1E70846BFE700BF3F420F0083
:101E100040787D0170B505460E464FF47A746B6AC2
:101E20005B6803F00103B34207D04FF47A7001F00E
:101E3000EFFC013CF3D1204670BD0120FCE700001F
:101E400070B5426A936913F0700F17D000230C4DE0
:101E5000936141F2900400EB4312224411794E0742
:101E600009D5890707D5416A55F823608E60117935
:101E700041F0040111710133032BECD170BD00BF9F
:101E8000404B000873B51D46436A16469A68D20750
:101E9000044609D59A6801219960C2F34002CDE950
:101EA00000650021FFF760FE636A9A68D1050BD5D3
:101EB0009A684FF480719960C2F34022CDE90065C1
:101EC00001212046FFF750FE636A9A68D2030BD5C2
:101ED0009A684FF480319960C2F34042CDE90065C1
:101EE00002212046FFF740FE04F58053D3F8DC00C2
:101EF00010B103681B699847204602B0BDE87040E6
:101F0000FFF79EBFF8B50446466A002977D106F16F
:101F10000C073868800775D006EB01153868D5F8CE
:101F2000B00110F0040FD5F8B0011ABFC00840F09E
:101F30000040400DA062D5F8B0C11CF0020F1CBFDC
:101F400040F08040A062D5F8B40106EB011100F02A
:101F50000F0084F83400D1F8B80184F82C00D1F8CF
:101F6000B801000A84F82D00D1F8B801000C84F8FB
:101F70002E00D1F8B801000E84F82F00D1F8BC0172
:101F800084F83000D1F8BC01000A84F83100D1F89F
:101F9000BC01000C84F83200D1F8BC11090E84F8A1
:101FA00033103821396004F1440004F1280104F1B0
:101FB000340551F8046B40F8046BA942F9D1098843
:101FC0000180C4E90E2321460023A4F8403051F8D3
:101FD000383B20461B6C984704F5805393F8D82073
:101FE000D3F8DC0042F0040283F8D82010B1036873
:101FF0001B6998472046BDE8F840FFF721BF06F16E
:10200000100786E7F8BD000010B5044600F05AFA44
:1020100002460B4652EA030102D0013A63F1000383
:102020000449086820B12146BDE81040FFF76ABFA7
:1020300010BD00BF284A0020F0B5302181F311887F
:10204000DFF848E000F583511831002441F2900C8C
:1020500000EB441565442E7977070ED4F6060CD5AF
:10206000D1E9007697429E4107D2466A5EF8247015
:10207000B7602E7946F004062E710134032C01F16D
:102080002001E5D1002383F31188F0BD404B000807
:1020900008B5302383F31188FFF7D2FE002383F3C2
:1020A000118808BD2DE9F041436A0446986800F0A4
:1020B000E050B0F1E05F0E4622D0F8B1302383F358
:1020C0001188002504F5845741F2900804EB45136C
:1020D00043441B791A0706D50135032D07F1200764
:1020E000F4D1012007E05B07F6D43946304600F012
:1020F00083FA0028F0D1002383F31188BDE8F08132
:102100000120FBE708B5302383F3118800F58050E8
:10211000C06EFFF725FB002383F3118843090CBF32
:102120000120002008BD0000F8B51D4600231370F3
:102130000F4606461446FFF7E5FF80F001003870B1
:1021400025B129463046FFF7ADFF2070F8BD0000ED
:102150002DE9B8410C4615461F46804600F0B2F9FD
:102160000B462178024609B9287850B14046FFF75E
:1021700063FFFFF78DFF3B462A462146FFF7D4FF5A
:102180000120BDE8B881000070B5302686F31188C3
:10219000174B1A6C42F000721A641A6A42F000720D
:1021A0001A621A6A22F000721A62002383F31188FD
:1021B00000F5805494F8D83013F0010516D1A9B178
:1021C00086F311880321132001F01EFA0321142045
:1021D00001F01AFA0321152001F016FA94F8D8300C
:1021E00043F0010384F8D83085F3118870BD00BF37
:1021F000003802402DE9F04700F5805588B095F889
:10220000E030012B04468846164600F28280824F59
:1022100057F823200AB947F82300D7F800A0C4F8DC
:102220001C8084F82060BAF1000F64D095F8E0308B
:10223000012B70D001212046FFF7A6FF302383F346
:102240001188626A136823F002031360626A1368DC
:1022500043F001031360636A00275F6187F311880D
:1022600001212046FFF7D6FD002800F09580E86E9A
:10227000FFF764FA04F58359BA4609F118092022D8
:1022800000216846FEF728FF02A8FFF759FCCDF8A9
:1022900018A06A4609EB07030DF1180E9446BCE836
:1022A0000300F44518605960624603F10803F5D154
:1022B000DCF80000186020379CF804201A71602FA9
:1022C000DDD195F8D8306FF38203002785F8D83038
:1022D0006A4641462046ADF80070ADF802708DF8B0
:1022E0000470FFF73BFD636A48BB4FF400421A607D
:1022F00008B0BDE8F08741F2E800FFF74FFB8146E8
:1023000010B15146FFF7C6FCC7F80090B9F1000FB5
:102310008CD10020ECE7386803681B6B98470146B6
:10232000002887D13868FFF72FFF386803683246E6
:102330005B684146984700287FF47CAFE9E761225B
:102340001A609DF802309DF803201B06120402F467
:10235000702203F040731343BDF80020C2F309025A
:1023600013439DF804201205022E02F4E0020CBF74
:102370004FF0004100211343626A0B43D361636A4B
:1023800013225A61626A136823F00103136039460D
:102390002046FFF73FFD08B9636AA6E795F8E030ED
:1023A00093BB616AD1F8002242F00102C1F8002219
:1023B000616AD1F8002222F47C5222F00E02C1F8A8
:1023C0000022616AD1F8002242F46062C1F8002262
:1023D000626AC2F81432626AC2F80432626A41F672
:1023E000FF71C2F80C12626AC2F84032626AC2F827
:1023F0004432636A0122C3F81C22626AD2F80032B6
:1024000023F00103C2F8003295F8D83043F00203FC
:1024100085F8D8306CE700BF284A002008B500F0E6
:1024200051F850EA0103024602D0421E61F1000158
:10243000044B186810B10B46FFF724FDBDE80840B7
:1024400001F0B8B8284A002008B50020FFF7DCFDED
:10245000BDE8084001F0AEB808B50120FFF7D4FD93
:10246000BDE8084001F0A6B800B59BB0EFF30981C4
:1024700068226846FEF71EFEEFF30583014B9B6B57
:10248000FEE700BF00ED00E008B5FFF7EDFF00003C
:1024900000B59BB0EFF3098168226846FEF70AFE9B
:1024A000EFF30583014B5B6BFEE700BF00ED00E03F
:1024B000FEE700000FB408B5029801F059F9FEE7F5
:1024C00001F06ABC01F04CBC0139C9B202299EBFBF
:1024D00000EBC1000023C0E901337047F8B51B8849
:1024E0005B0705460E4615D4044600F11807BC42AA
:1024F00010D0636853B12B682846DB6B9847A368FC
:10250000C1B23246606898470834F0E7A368002BF0
:10251000F1D1F9E70120F8BD73B56C4684E80600F7
:10252000014600224E68D5B26EB98E685EB900EBE6
:10253000C200021D94E80300013582E803001D700B
:10254000012002B070BD0132032A01F10801E9D176
:102550000020F6E72DE9F04F89B00446BDF8487039
:102560000E46054600F118084FF0000907F0040771
:102570004FF0000A4FF0000BA84538D06B680BB93C
:10258000AB684BB157B923682046DB6B9847AB6803
:10259000C1B23246686898470835EDE7B9F1000FD7
:1025A000FAD1CDE900ABADF80890334603AA06F1A5
:1025B000080E186859689446ACE803000833734560
:1025C0006246F6D11868CCF800009B88ACF804305D
:1025D000FFF778FF0423ADF808302368CDE9000148
:1025E0001B6C6946204698474FF00109D4E701204B
:1025F00009B0BDE8F08F000030B503680968DD0F51
:10260000B5EBD17F23F0604421F060424FEAD170F6
:102610000BD0002BB8BFA40C0029B8BF920C944279
:1026200002D034BF0120002030BD944205D1C1F357
:102630008070C3F380738342F6D194422CBF002094
:102640000120F1E72DE9F041456A15B94162BDE885
:10265000F0814B6823F06047C3F38A464FEAD37E8C
:10266000C3F3807816EA230638BF3E46AC462B46B5
:102670005A68BEEBD27F22F060440AD0002A18DAF2
:10268000A40CB44217D19D420FD10D60DEE7134672
:10269000EEE7A74207D102F08044C2F380724245C0
:1026A0000BD054B1EFE708D2EDE7CCF800100B6087
:1026B000CDE7B44201D0B442E5D81A689C46002A5E
:1026C000E5D11960C3E700002DE9F047089D01F04E
:1026D00007044FEAD508224405F0070500EBD100B6
:1026E0004FF47F49944201D1BDE8F08704F0070719
:1026F00005F0070A57453E4638BF5646C6F108065C
:10270000111B8E4228BF0E46E10808EBD50E415C36
:1027100013F80EC0B94029FA06F721FA0AF1FFB200
:102720008CEA010147FA0AF739408CEA010C03F8F8
:102730000EC034443544D5E780EA0120082341F235
:10274000210201B24000002980B203F1FF33B8BF7B
:10275000504013F0FF03F4D17047000038B50C4629
:102760008D18A54200D138BD14F8011BFFF7E4FF16
:10277000F7E7000042684AB11368436043898189E2
:1027800001339BB29942438138BF83811046704721
:1027900070B588B0202204460D4668460021FEF739
:1027A0009BFC20460495FFF7E5FF024658B16B46B7
:1027B000054608AE1C4603CCB44228606960234637
:1027C00005F10805F6D1104608B070BD082817D9E4
:1027D00009280CD00A280CD00B280CD00C280CD0BF
:1027E0000D280CD00E2814BF4020302070470C203C
:1027F0007047102070471420704718207047202021
:1028000070470000082817D90C280CD910280CD9BB
:1028100014280CD918280CD920280CD930288CBFA2
:102820000F200E207047092070470A2070470B20A8
:1028300070470C2070470D20704700002DE9F843C9
:10284000078C072F04461ED9D0E9029800254FF6C1
:10285000FF73C5F12006A5F1200029FA05F108FA59
:1028600006F628FA00F031430143C9B21846FFF7D3
:1028700063FF0835402D0346EBD1E1693A46BDE8D8
:10288000F843FFF76BBF4FF6FF70BDE8F883000019
:1028900010B54B6823B9CA8A63F30902CA8210BD16
:1028A00004691A681C600361C38A013BC3824A60E1
:1028B000EFE700002DE9F84F1D46CB8A0F46C3F322
:1028C00009010529814692460B4630D00020AAB264
:1028D00007F11A049EB2042E1FFA80F80FD8904513
:1028E00003F1010306D3FB8A0A4462F30903FB8266
:1028F00001201AE01AF80060E6540130EAE790453A
:10290000F1D2A1F1050B1C237C68BBFBF3F203FBA6
:1029100012BB1FFA8BF6002C45D14846FFF72AFF61
:10292000044638B978606FF00200BDE8F88F4FF0C8
:102930000008E6E7002606607860ADB24FF0000BB5
:10294000454510D90AEB0803221D13F8011B9155C8
:10295000B1B208F101081B291FFA88F82BD04545B0
:1029600006F10106F1D8FB8AC3F30902154465F3A9
:102970000903BCE7013292B21C462368002BF9D14F
:102980006B1F0B441C21B3FBF1F301339BB29A4242
:10299000D3D2BBF1000FD0D14846FFF7EBFE20B9F0
:1029A000C4F800B0BFE70122E7E7C0F800B05E4618
:1029B00020600446C1E74545D5D94846FFF7DAFE11
:1029C00008B92060AFE7C0F800B0002620600446D8
:1029D000B6E700002DE9F04F2DED028B1C4683B0C9
:1029E0005B69019207468846002B00F0A780238C84
:1029F0002BB1E269002A00F0A180072B35D807F13E
:102A00000C00FFF7B7FE054638B96FF002052846FF
:102A100003B0BDEC028BBDE8F08F14220021FEF75D
:102A20005BFB228CE16905F10800FEF743FB208C7B
:102A3000013080B2FFF7E6FEFFF7C8FE013880B232
:102A40002084013028746369228C1B782A4403F0A7
:102A50001F0363F03F0348F000411372384669607A
:102A60002946FFF7EFFD0125D1E702339BB207228C
:102A7000C18A0633B3FBF2F3828A521A9BB292B236
:102A80009342C2D800F10C034FF0000908EE103A4F
:102A90004FF0800A4E464D4618EE100AFFF76AFEC8
:102AA00083460028B1D014220021FEF715FB002E2A
:102AB0003AD1019BABF8083002220BF1080E1FFA45
:102AC00082FC0CF10100BCF1060F218C80B201D810
:102AD0008E422BD3FFF796FEFFF778FE62691278DD
:102AE000013802F01F028E4208BF4FF0400A42EA4E
:102AF00049121BFA80F14AEA020A013048F000420A
:102B000081F808A08BF81000CBF80420594638460D
:102B1000FFF798FD238C0135B3422DB289F00109EE
:102B20004FF0000AB8D172E70022C6E7E169895D7B
:102B30000EF802100136B6B20132C0E76FF001059F
:102B400065E70000F8B515460E4630220021044620
:102B50001F46FEF7C1FA069B6360B5F5001F079B91
:102B6000A76034BF6A094FF6FF72A36297B2E661AD
:102B700004F1100000239A4206D800230360A782C4
:102B8000E3822383E360F8BD0660013330462036DC
:102B9000F1E7000003781BB94BB2002BC8BF0170EE
:102BA0007047000000787047F8B50C46C9690746C1
:102BB00011B9238C002B37D1257E1F2D34D83878BE
:102BC00028BB228C072A2CD8268A36F003032BD167
:102BD0004FF6FF70FFF7C2FD20F001003102400404
:102BE00041EA0561400C41EA40254FF6FF72234659
:102BF00029463846FFF7EEFE002807DD62691378A4
:102C00000133DBB21F2B88BF00231370F8BD218A6C
:102C10002D0645EA012505432046FFF70FFE024633
:102C2000E5E76FF00300F1E76FF00100EEE7000069
:102C300070B58AB0044616460021282268461D4613
:102C4000FEF74AFABDF83830ADF810300F9B059307
:102C50009DF840308DF81830119B07936946BDF8F8
:102C60004830ADF820302046CDE90265FFF79CFFE3
:102C70000AB070BD2DE9F041D36905460C461646F1
:102C80000BB9138C5BBB377E1F2F28D895F80080BB
:102C9000B8F1000F26D03046FFF7D0FD337821027F
:102CA00041EAC33141EA0801338A41EA076141EA56
:102CB00003410246334641F080012846FFF78AFE71
:102CC00000280ADD3378012B07D1726913780133AC
:102CD000DBB21F2B88BF00231370BDE8F0816FF0BB
:102CE0000100FAE76FF00300F7E70000F0B58BB0E2
:102CF00004460D4617460021282268461E46FEF768
:102D0000EBF99DF84C305A1E534253418DF8003078
:102D10009DF84030ADF81030119B05939DF8483078
:102D20008DF81830149B07936A46BDF85430ADF8FF
:102D3000203029462046CDE90276FFF79BFF0BB0F5
:102D4000F0BD0000406A00B104307047436A1A6861
:102D5000426202691A600361C38A013BC382704701
:102D60002DE9F041D0F82080194E14461D46414609
:102D7000002709B9BDE8F081D1E90223A21A65EB69
:102D80000303964277EB03031ED2036A8B420DD1F5
:102D9000FFF77EFD036A1B68036203690B60C38A49
:102DA0000161016A013BC3828846E2E7FFF770FDDB
:102DB0000B68C8F8003003690B60C38A0161013BEE
:102DC000C382D8F80010D4E788460968D1E700BF6D
:102DD00080841E002DE9F04F8BB00D46DDF8509039
:102DE00014469B468046002800F01981B9F1000F77
:102DF00000F01581531E3F2B00F21181012A03D1EF
:102E0000BBF1000F40F00B810023CDE90833B8F887
:102E10001430B5EBC30F4FEAC30703D300200BB048
:102E2000BDE8F08F2B199F42D8F80C303ABF7F1BBA
:102E3000FFB227461BB9D8F81030002B7AD0272DC7
:102E40004ED8C5F12806B7424FF000032CBFF6B2AA
:102E50003E4600932946D8F8080008AB3246FFF7F3
:102E600033FCA7EB060A35445FFA8AFAB8F8143047
:102E700003F10053053BDB000493D8F80C300393B7
:102E80002821039B13B1BAF1000F2CD1D8F8100000
:102E900040B1BAF1000F05D0009608AB5246691A4E
:102EA000FFF712FC38B2002FB8D066070AD00AAB81
:102EB00003EBD401624211F8083C02F0070213410F
:102EC00001F8083C082C3CD9102C40F2B580202C8D
:102ED00040F2B780BBF1000F00F09C80082334E083
:102EE000BA460026C2E7049BE02B28BFE0230693E6
:102EF0000B44AB42059314D95A1B03980096924594
:102F000034BF5246D2B2691A08AB04300792FFF7B9
:102F1000DBFB079A1644AAEB020A1544F6B25FFAE5
:102F20008AFA049B069A05999B1A0493039B1B68D3
:102F30000393A6E70093D8F8080008AB3A46294661
:102F4000AEE7BBF1000F13D00123B4EBC30F6CD07D
:102F5000082C12D89DF82030621E23FA02F2D50701
:102F600006D54FF0FF3202FA04F423438DF82030E7
:102F70009DF8203089F8003051E7102C12D8BDF8A8
:102F80002030621E23FA02F2D10706D54FF0FF323D
:102F900002FA04F42343ADF82030BDF82030A9F83C
:102FA00000303CE7202C0FD80899631E21FA03F368
:102FB000DA0705D54FF0FF3202FA04F40C43089407
:102FC000089BC9F800302AE7402C2BD0DDE90865C2
:102FD000611EC4F12102A4F1210326FA01F105FAD0
:102FE00002F225FA03F311431943CB0712D501224C
:102FF000A4F12003C4F1200102FA03F322FA01F143
:10300000A240524243EA010363EB430332432B43A2
:10301000CDE90823DDE90823C9E90023FFE66FF0C5
:103020000100FCE66FF00800F9E6082CA0D9102C8E
:10303000B3D9202CEED8C3E7BBF1000FADD00223EB
:1030400083E7BBF1000FBBD004237EE730B5012A34
:10305000144638BF0124402C85B028BF40240025E9
:10306000012ACDE9025518D81B788DF8083063077E
:103070000AD004AB03EBD405624215F8083C02F019
:103080000702934005F8083C0091034622460021C0
:1030900002A8FFF719FB05B030BD082AE4D9102AB1
:1030A00003D81B88ADF80830E1E7202A8DBFD3E9AB
:1030B00000231B680293CDE90223D8E710B5CB6843
:1030C0001BB98B600B618B8210BD04691A681C6090
:1030D0000361C38A013BC382CA60F0E703064CBFA9
:1030E000C0F3C0300220704708B50246FFF7F6FF74
:1030F000022806D15306C2F30F2001D100F00300CD
:1031000008BDC2F30740FBE72DE9F04F93B0CDE9CE
:1031100003230A6804461046FFF7E0FF022814BFA5
:10312000C2F306260026002A0D46824680F2F78169
:1031300012F0C04940F0F381097B002900F0EF81D3
:10314000022803D02378B34240F0EC81C2F3046339
:103150000693104602F07F030593FFF7C5FF059B1A
:1031600029444FEA834848EA0A4848EA4668CE7844
:1031700000230022CDE90823F309834648EA00082A
:10318000029367D0059B009302466768534608A9DF
:103190002046B847002800F0C881276A4FB9414649
:1031A00004F10C00FFF7F4FA074690B96FF0020043
:1031B00054E03B6998450DD03F68002FF9D1414656
:1031C00004F10C00FFF7E4FA07460028EED0236A6A
:1031D0003B60276297F817C006F01F08CCF3840CF9
:1031E000ACEB08001FFA80FE0028B8BF0EF12000EB
:1031F000A8EB0C031FFA83FED7E90221B8BF00B287
:10320000002B0793BEBF0EF120031BB2079352EAB7
:10321000010338D0039BDFF824E39A1A049B4FF094
:10322000000C63EB010196457CEB01032BD36B7B18
:1032300097F81AE0734519D1029B002B78D001282A
:1032400021DC7868F8B9DFF8F0C2944570EB01032F
:1032500016D337E0276A27B96FF00C0013B0BDE82A
:10326000F08F3B699845B5D03F68F4E7B24890428B
:103270007CEB010301D30020F0E7029B002BFAD086
:10328000079B0F2B17DCFA7DB30002F0030203F05B
:103290007C031343FB7539462046FFF7F9FA6B7B35
:1032A000BB76029B3BB9FB7DC3F38402013262F320
:1032B0008603FB75D0E76A7BBB7E9A42DBD1029B1B
:1032C000002B35D0B309022B32D0039BBB60049B8B
:1032D000FB60142200210DA8FDF7FEFE039B0A935C
:1032E000049B0B932B1D0C932B7BADF83EB0013B45
:1032F000DBB2ADF83C30069B8DF84230059B8DF873
:10330000433094F82C308DF840A083F001038DF801
:1033100044308DF84180A3680AA920469847FB7D78
:10332000C3F38403013303F01F039B02FB82A2E774
:10333000FB7DC6F34012B2EBD31F40F0F980C3F31C
:103340008403434540F0FC80029A2B7BB609002A97
:1033500052D016F0010661D1032B40F2F480039B9A
:10336000BB60049BFB60FB8A66F30903FB822B7B3B
:10337000AE1D033BDBB23246394604F10C00FFF7C9
:1033800099FA00280CDA39462046FFF781FAFB7DCE
:10339000C3F38403013303F01F039B02FB8205E7A1
:1033A000DDE90884AB883B834FF6FF73C9F1200049
:1033B000A9F1200228FA09F104FA00F0014324FAE5
:1033C00002F211431846C9B2FFF7B6F909F108092C
:1033D000B9F1400F0346E9D1B8822A7B033AD2B251
:1033E0003146FFF7BBF9FB7DB882DA43C2F3C01266
:1033F00062F3C713FB753EE786B92E1D013BDBB2B6
:103400003246394604F10C00FFF754FA0028BADBC3
:103410002A7BB88A013AD2B23146E2E7F98AC1F38F
:103420000901013B0429DAB25BD8281D002307F10A
:103430001B069A4208D910F801CB06F801C00131E9
:1034400001330529DBB2F4D103990A9104990B9158
:10345000934207F11B010C9138BF043379680D9139
:1034600034BF55FA83F300230E93FB8AADF83EB0C8
:10347000C3F309031A44069B8DF84230059B8DF86F
:10348000433094F82C30ADF83C2083F001038DF8E4
:10349000443000238DF840A08DF841807B602A7B6A
:1034A000B88A013A291DFFF759F93B8BB88283424C
:1034B00003D1A3680AA92046984720460AA9FFF726
:1034C000FDFDFB7DBA8AC3F38403013303F01F03C0
:1034D0009B02FB823B8B9A420CBF00206FF01000D6
:1034E000BCE67B68002BAFD0052001E01C303346E2
:1034F0001E68002EFAD1091A081D2E1D184401EB72
:10350000090CBCF11B0F5FFA89F39DD89A429BD935
:1035100016F8013B00F8013B09F10109EFE76FF0F4
:1035200009009BE66FF00A0098E66FF00B0095E645
:103530006FF00D0092E600BF40420F0080841E0035
:103540006FF00E008AE66FF00F0087E6EFF3098355
:1035500005494A6B22F001024A63683383F3098804
:10356000002383F31188704700EF00E0302080F3E0
:10357000118862B60C4B0D4AD96821F4E061090448
:10358000090C0A43DA60D3F8FC20094942F0807242
:10359000C3F8FC200A6842F001020A602022DA77B0
:1035A00083F82200704700BF00ED00E00003FA0539
:1035B000001000E010B5302383F311880E4B5B68D8
:1035C00013F4006314D0F1EE103AEFF30984683C71
:1035D0004FF08073E361094BDB6B236684F309884A
:1035E00000F090F810B1064BA36110BD054BFBE74E
:1035F00083F31188F9E700BF00ED00E000EF00E081
:103600003F0300084203000800F1604303F56143F3
:103610000901C9B283F80013012200F01F039A4088
:1036200043099B0003F1604303F56143C3F8802124
:103630001A60704700230375826803691B689968E4
:103640009142FBD25A680360426010605860704734
:1036500000230375826803691B6899689142FBD84F
:103660005A680360426010605860704708B50846A9
:10367000302383F311880B7D032B05D0042B0DD051
:103680002BB983F3118808BD8B6900221A604FF0B3
:10369000FF338361FFF7CEFF0023F2E7D1E9003269
:1036A00013605A60F3E70000FFF7C4BF054BD96809
:1036B0000875186802681A60536001220275D860A4
:1036C000FCF728BE384A002030B50C4BDD684B1C97
:1036D00087B004460FD02B46094A684600F046F9E9
:1036E0002046FFF7E3FF009B13B1684600F048F95E
:1036F000A86907B030BDFFF7D9FFF9E7384A0020C5
:103700006D360008044B1A68DB6890689B68984225
:1037100094BF002001207047384A0020084B10B5A4
:103720001C68D86822681A60536001222275DC6028
:10373000FFF78EFF01462046BDE81040FCF7EABDCA
:10374000384A002038B5074C0749084801230025AE
:103750002370656000F024FC0223237085F3118838
:1037600038BD00BFA04C00209C4B0008384A002008
:1037700008B572B6044B186500F0E2FA00F08AFB57
:10378000024B03221A70FEE7384A0020A04C0020AA
:1037900000F02CB98B60022308618B8208467047C9
:1037A0008368A3F1840243F8142C026943F8442C83
:1037B000426943F8402C094A43F8242CC26843F874
:1037C000182C022203F80C2C002203F80B2C044ABC
:1037D00043F8102CA3F12000704700BF2D03000810
:1037E000384A002008B5FFF7DBFFBDE80840FFF7C7
:1037F0005BBF0000024BDB6898610F20FFF756BFEC
:10380000384A0020302383F31188FFF7F3BF00000C
:1038100008B50146302383F311880820FFF754FFD1
:10382000002383F3118808BD064BDB6839B1426879
:1038300018605A60136043600420FFF745BF4FF0E3
:10384000FF307047384A00200368984206D01A6853
:103850000260506099611846FFF726BF704700006C
:1038600010B503689C68A2420CD85C688A600B6043
:103870004C602160596099688A1A9A604FF0FF3352
:10388000836010BD1B68121BECE700000A2938BFDB
:103890000A2170B504460D460A26601900F07AFB2D
:1038A00000F066FB041BA54203D8751C2E46044697
:1038B000F3E70A2E04D9BDE87040012000F0B0BB48
:1038C00070BD0000F8B5144B0D46D96103F110012D
:1038D00041600A2A1969826038BF0A220160486083
:1038E0001861A818144600F047FB0A2700F040FBB7
:1038F000431BA342064606D37C1C281900F04AFB52
:1039000027463546F2E70A2F04D9BDE8F8400120E2
:1039100000F086BBF8BD00BF384A0020F8B5064667
:103920000D4600F025FB0F4A134653F8107F9F42C7
:1039300006D12A4601463046BDE8F840FFF7C2BF2F
:10394000D169BB68441A2C1928BF2C46A34202D95E
:103950002946FFF79BFF224631460348BDE8F84061
:10396000FFF77EBF384A0020484A002010B4C0E963
:10397000032300235DF8044B4361FFF7CFBF000032
:1039800010B5194C236998420DD0D0E900328168F6
:1039900013605A609A680A449A60002303604FF0EB
:1039A000FF33A36110BD2346026843F8102F536014
:1039B0000022026022699A4203D1BDE8104000F063
:1039C000E3BA936881680B44936000F0D1FA2269EE
:1039D000E1699268441AA242E4D91144BDE810405A
:1039E000091AFFF753BF00BF384A00202DE9F047FE
:1039F000DFF8BC8008F110072C4ED8F8105000F00A
:103A0000B7FAD8F81C40AA68031B9A423ED814445F
:103A1000D5E900324FF00009C8F81C4013605A6025
:103A2000C5F80090D8F81030B34201D100F0ACFADC
:103A300089F31188D5E9033128469847302383F369
:103A400011886B69002BD8D000F092FA6A69A0EB5C
:103A500004094A4582460DD2022000F0E1FA002214
:103A6000D8F81030B34208D151462846BDE8F04797
:103A7000FFF728BF121A2244F2E712EB090938BFF8
:103A80004A4629463846FFF7EBFEB5E7D8F810302E
:103A9000B34208D01444211AC8F81C00A960BDE83C
:103AA000F047FFF7F3BEBDE8F08700BF484A0020AB
:103AB000384A002038B500F05BFA054AD2E90845DB
:103AC000031B181945F10001C2E9080138BD00BF08
:103AD000384A002000207047FEE7000070470000D1
:103AE0004FF0FF3070470000BFF34F8F024AD3689A
:103AF000DB03FCD4704700BF003C024008B5094B13
:103B00001B7873B9FFF7F0FF074B1A69002ABFBF94
:103B1000064A5A6002F188325A601A6822F48062BA
:103B20001A6008BDA84C0020003C024023016745F4
:103B300008B50B4B1B7893B9FFF7D6FF094B1A69F1
:103B400042F000421A611A6842F480521A601A6800
:103B500022F480521A601A6842F480621A6008BD2A
:103B6000A84C0020003C02400728F0B516D80C4CA9
:103B70000C4923787BB90C4D0E4608234FF00062A8
:103B800055F8047B46F8042B013B13F0FF033A443D
:103B9000F6D10123237051F82000F0BD0020FCE78E
:103BA000CC4C0020AC4C0020A84B0008014B53F833
:103BB00020007047A84B000808207047072810B560
:103BC000044601D9002010BDFFF7CEFF064B53F885
:103BD00024301844C21A0BB90120F4E712680132EC
:103BE000F0D1043BF6E700BFA84B0008072810B54A
:103BF000044621D8FFF778FFFFF780FF0F4AF32331
:103C0000D360C300DBB243F4007343F002031361DB
:103C1000136943F480331361FFF766FFFFF7A4FFD6
:103C2000074B53F8241000F031F9FFF781FF2046CD
:103C3000BDE81040FFF7C2BF002010BD003C0240AD
:103C4000A84B0008F8B512F00103144642D18518BC
:103C50002E4A954257D82E4B1B6813F0010352D0C1
:103C60002C4DFFF74BFFF323EB60FFF73DFF40F2D6
:103C70000127032C15D824F001046618254C401A9E
:103C800040F20117B142236900EB010524D123F072
:103C900001032361FFF74CFF0120F8BD043C043011
:103CA000E7E78307E7D12B6923F440732B612B6986
:103CB0003B432B6151F8046B0660BFF34F8FFFF756
:103CC00013FF03689E42E9D02B6923F001032B61A7
:103CD000FFF72EFF0020E0E723F440732361236900
:103CE0003B4323610B882B80BFF34F8FFFF7FCFE14
:103CF0002D8831F8023BADB2AB42C3D0236923F02B
:103D000001032361E4E71846C7E700BF0000080885
:103D100000380240003C0240084908B50B7828B141
:103D20001BB9FFF7EBFE01230B7008BD002BFCD085
:103D3000BDE808400870FFF7FBBE00BFA84C00209C
:103D40000149024800F0A4B800FF03000001002070
:103D50000846114600F07CBE084600F08FBE000009
:103D600038B5EFF311859DB9EFF30584C4F308046A
:103D7000302334B183F31188FFF79CFE85F311885B
:103D800038BD83F31188FFF795FE84F3118838BDA1
:103D9000BDE83840FFF78EBE38B5FFF7E1FF114CA4
:103DA000114AC00840EA4170A0FB025EC908A0FBAE
:103DB000040C1CEB050CA1FB04404FF000035B411D
:103DC000A1FB02121CEB040C43EB000011EB0E01F3
:103DD00042F10002411842F10000090941EA007075
:103DE00038BD00BFCFF753E3A59BC42010B50244F4
:103DF000064BD2B2904200D110BD441C00B253F821
:103E0000200041F8040BE0B2F4E700BF5028004066
:103E10000F4B30B51C6F240407D41C6F44F400749E
:103E20001C671C6F44F400441C670A4C236843F46D
:103E3000807323600244084BD2B2904200D130BD5F
:103E4000441C00B251F8045B43F82050E0B2F4E7A0
:103E500000380240007000405028004007B50122A1
:103E600001A90020FFF7C2FF019803B05DF804FB31
:103E700013B50446FFF7F2FFA04205D0012201A9C5
:103E800000200194FFF7C4FF02B010BD704700008E
:103E90007047000070470000074B45F255521A600A
:103EA00003225A6040F2FF729A604CF6CC421A60CC
:103EB000024B01221A70704700300040D44C0020A1
:103EC000034B1B781BB1034B4AF6AA221A607047BA
:103ED000D44C002000300040034B1A681AB9034A42
:103EE000D2F874281A607047D04C0020003002408D
:103EF000024B4FF08072C3F87428704700300240C4
:103F000008B5FFF7E9FF024B1868C0F3407008BD21
:103F1000D04C002008B5FFF7DFFF024B1868C0F354
:103F2000007008BDD04C002070470000FEE7000084
:103F30000A4B0B480B4A90420BD30B4BDA1C121A5C
:103F4000C11E22F003028B4238BF00220021FDF780
:103F5000C3B853F8041B40F8041BECE7604D00089D
:103F6000C44F0020C44F0020C44F002000F0CAB846
:103F70004FF08043586A70474FF0804300225863E7
:103F80001A610222DA6070474FF080430022DA6043
:103F9000704700004FF0804358637047FEE7000011
:103FA00070B51B4B01630025044686B058608562DE
:103FB0000E46FFF7DBFA04F11003C4E904334FF0B7
:103FC000FF33C4E90635C4E90044A560E562FFF7A4
:103FD000CFFF2B460246C4E9082304F134010D4A01
:103FE000256580232046FFF7D5FB0123E0600A4AC0
:103FF0000375009272680192B268CDE90223074B03
:104000006846CDE90435FFF7EDFB06B070BD00BF93
:10401000A04C0020C84B0008CD4B00089D3F000875
:10402000024AD36A1843D062704700BF384A002062
:104030004B6843608B688360CB68C3600B694361E6
:104040004B6903628B6943620B6803607047000031
:1040500008B5234B23481A6942F0FF021A611A6916
:1040600022F0FF021A611A691A6B42F0FF021A630A
:104070001A6D42F0FF021A651B4A1B6D1146FFF7CD
:10408000D7FF02F11C0100F58060FFF7D1FF02F1BC
:10409000380100F58060FFF7CBFF02F1540100F515
:1040A0008060FFF7C5FF02F1700100F58060FFF747
:1040B000BFFF02F18C0100F58060FFF7B9FF02F14C
:1040C000A80100F58060FFF7B3FF02F1C40100F51D
:1040D0008060FFF7ADFFBDE8084000F08DB800BF7D
:1040E0000038024000000240D44B000808B500F040
:1040F00019FAFFF727FBBDE80840FFF7EDBE000007
:10410000704700000F4B1A6C42F001021A641A6EDD
:1041100042F001021A660C4A1B6E936843F00103D9
:1041200093604FF0804331229A624FF0FF32DA629F
:1041300000229A615A63DA605A6001225A611A6059
:10414000704700BF00380240002004E04FF080427A
:1041500008B51169D3680B40D9B2C9439B071161F7
:1041600007D5302383F31188FFF712FB002383F375
:10417000118808BD1E4B1A6962F0FF021A611A69A4
:10418000D2B21A614FF0FF301A695A6958610021A2
:104190005A6959615A691A6A62F080521A621A6A37
:1041A00002F080521A621A6A5A6A58625A6A59624E
:1041B0005A6A1A6C42F080521A641A6E42F08052A7
:1041C0001A661A6E0B4A106840F480701060186FFF
:1041D00000F44070B0F5007F1EBF4FF480301867C8
:1041E0001967536823F40073536000F073B900BF7C
:1041F00000380240007000403B4B3C4A1A643C4A85
:104200004FF4404111601A6842F001021A601A68C6
:104210009007FCD59A6822F003029A60324B9A68A4
:1042200012F00C02FBD1196801F0F90119609A60D3
:104230001A6842F480321A601A689103FCD55A6FEA
:1042400042F001025A67284B5A6F9207FCD5294A5F
:104250005A601A6842F080721A60254A53685804FE
:10426000FCD5214B1A689101FCD5234AC3F8842060
:104270001A6842F080621A601A681201FCD51F4A5F
:104280009A600322C3F88C204FF00062C3F8942098
:104290001B4B1A681B4B9A421B4B21D11B4A1168BE
:1042A0001B4A91421CD140F203121A60164A13684D
:1042B00003F00F03032BFAD10B4B9A6842F0020272
:1042C0009A609A6802F00C02082AFAD15A6C42F4F9
:1042D00080425A645A6E42F480425A665B6E70475E
:1042E00040F20372E1E700BF003802400004001012
:1042F00000700040041940020830002400948838FF
:10430000002004E011640020003C024000ED00E0C9
:1043100041C20F41074A08B5536903F001035361D5
:1043200023B1054A13680BB150689847BDE80840AF
:10433000FFF740B9003C0140D84C0020074A08B5BF
:10434000536903F00203536123B1054A93680BB12B
:10435000D0689847BDE80840FFF72CB9003C014001
:10436000D84C0020074A08B5536903F00403536191
:1043700023B1054A13690BB150699847BDE808405D
:10438000FFF718B9003C0140D84C0020074A08B597
:10439000536903F00803536123B1054A93690BB1D4
:1043A000D0699847BDE80840FFF704B9003C0140D8
:1043B000D84C0020074A08B5536903F01003536135
:1043C00023B1054A136A0BB1506A9847BDE808400B
:1043D000FFF7F0B8003C0140D84C0020164B10B558
:1043E0005C6904F478725A61A30604D5134A936A8F
:1043F0000BB1D06A9847600604D5104A136B0BB115
:10440000506B9847210604D50C4A936B0BB1D06BC7
:104410009847E20504D5094A136C0BB1506C9847D4
:10442000A30504D5054A936C0BB1D06C9847BDE841
:104430001040FFF7BFB800BF003C0140D84C00203F
:10444000194B10B55C6904F47C425A61620504D5CD
:10445000164A136D0BB1506D9847230504D5134AC6
:10446000936D0BB1D06D9847E00404D50F4A136EDD
:104470000BB1506E9847A10404D50C4A936E0BB152
:10448000D06E9847620404D5084A136F0BB1506F81
:104490009847230404D5054A936F0BB1D06F984712
:1044A000BDE81040FFF786B8003C0140D84C002022
:1044B00008B5034800F0E8F8BDE80840FFF77AB80F
:1044C000584D002008B5FFF741FEBDE80840FFF752
:1044D00071B80000062108B50846FFF795F80621D7
:1044E0000720FFF791F806210820FFF78DF8062135
:1044F0000920FFF789F806210A20FFF785F8062131
:104500001720FFF781F806212820FFF77DF8072103
:104510001C20FFF779F8BDE808400C212620FFF7A2
:1045200073B8000008B5FFF725FE00F07BF800F037
:104530003DF8FFF7E5FDBDE80840FFF717BD0000B7
:10454000026843681143016003B1184770470000D7
:10455000143000F0C5B900004FF0FF33143000F004
:10456000BFB90000383000F03BBA00004FF0FF3315
:10457000383000F035BA0000143000F08BB900007C
:104580004FF0FF31143000F085B90000383000F0F2
:10459000E5B900004FF0FF32383000F0DFB900001D
:1045A000012914BF6FF013000020704700F058B8C5
:1045B00037B515460E4A026000224260C0E9022269
:1045C0000122044602740B46009000F15C014FF496
:1045D0008072143000F034F900942B464FF480724E
:1045E00004F5AE7104F1380000F0ACF903B030BD51
:1045F000B44C000838B5C36904460D461BB9042104
:104600000844FFF79DFF294604F1140000F026F945
:10461000002806DA201D4FF40061BDE83840FFF79E
:104620008FBF38BD0023054A19460133102BC2E95C
:10463000001102F10802F8D1704700BFD84C0020E9
:10464000026843681143016003B1184770470000D6
:10465000024AD36843F0C003D3607047004400406F
:1046600010B5054C054A00212046FFF7A1FF044A7A
:10467000044BC4E9972310BD584D00205146000853
:104680000044004040787D012DE9F041D0F85C62A3
:10469000F7683368DA0504469DB20DD5302383F3FD
:1046A00011884FF480610430FFF7CAFF6FF4807304
:1046B0003360002383F31188302383F3118804F1DE
:1046C000040815F02F033AD183F31188380615D565
:1046D000290613D5302383F3118804F1380000F044
:1046E00065F900284EDA0821201DFFF7A9FF4FF6D3
:1046F0007F733B40F360002383F311887A0616D55D
:104700006B0614D5302383F31188D4E913239A421E
:104710000AD1236C43B127F040073F041021201D2C
:104720003F0CFFF78DFFF760002383F31188D4F867
:104730006822D36843B3BDE8F041106918472B07DE
:1047400014D015F0080F0CBF00214FF48071E8075A
:1047500048BF41F02001AA0748BF41F040016B0764
:1047600048BF41F080014046FFF76AFFAD0673681D
:1047700005D594F8641220461940FFF73BFF3568D1
:10478000ADB29EE77060B6E7BDE8F081F8B51546BA
:1047900082680669AA420B46816938BF8568761A25
:1047A000B54204460BD218462A46FCF783FCA3699F
:1047B0002B44A361A3685B1BA3602846F8BD0CD9FA
:1047C00018463246FCF776FCAF1BE1683A463044A7
:1047D000FCF770FCE3683B44EBE718462A46FCF71D
:1047E00069FCE368E5E7000083689342F7B5154686
:1047F000044638BF8568D0E90460361AB5420BD24A
:104800002A46FCF757FC63692B446361A36828467A
:104810005B1BA36003B0F0BD0DD932460191FCF7DC
:1048200049FC0199E068AF1B3A463144FCF742FC71
:10483000E3683B44E9E72A46FCF73CFCE368E4E72D
:1048400010B50A440024C361029B8460C0E90000E3
:10485000C0E90511C1600261036210BD08B5D0E96D
:104860000532934201D1826882B982680132826046
:104870005A1C42611970D0E904329A4224BFC368BD
:1048800043610021FEF7E0FF002008BD4FF0FF303C
:10489000FBE7000070B5302304460E4683F3118811
:1048A000A568A5B1A368A269013BA360531CA361DD
:1048B00015782269934224BFE368A361E3690BB1D1
:1048C00020469847002383F31188284607E03146A5
:1048D0002046FEF7A9FF0028E2DA85F3118870BDB3
:1048E0002DE9F74F04460E4617469846D0F81C901F
:1048F0004FF0300A8AF311884FF0000B154665B16E
:104900002A4631462046FFF741FF034660B941463B
:104910002046FEF789FF0028F1D0002383F3118899
:10492000781B03B0BDE8F08FB9F1000F03D0019000
:104930002046C847019B8BF31188ED1A1E448AF369
:104940001188DCE7C0E90511C160C3611144009B17
:104950008260C0E90000016103627047F8B5044657
:104960000D461646302383F31188A768A7B1A368C4
:10497000013BA36063695A1C62611D70D4E9043273
:104980009A4224BFE3686361E3690BB1204698470C
:10499000002080F3118807E031462046FEF744FFEF
:1049A0000028E2DA87F31188F8BD0000D0E905237A
:1049B0009A4210B501D182687AB982680132826068
:1049C0005A1C82611C7803699A4224BFC3688361C0
:1049D0000021FEF739FF204610BD4FF0FF30FBE706
:1049E0002DE9F74F04460E4617469846D0F81C901E
:1049F0004FF0300A8AF311884FF0000B154665B16D
:104A00002A4631462046FFF7EFFE034660B941468D
:104A10002046FEF709FF0028F1D0002383F3118818
:104A2000781B03B0BDE8F08FB9F1000F03D00190FF
:104A30002046C847019B8BF31188ED1A1E448AF368
:104A40001188DCE70B460146184600F009B8000063
:104A5000024B0A4601461868FFF77AB91C2300206A
:104A600010B5054C13462CB10A4601460220AFF39F
:104A7000008010BD2046FCE700000000024B01460C
:104A80001868FFF769B900BF1C23002010B5013971
:104A90000244904201D1002005E0037811F8014F53
:104AA000A34201D0181B10BD0130F2E72DE9F041FF
:104AB000A3B1C91A17780144044603F1FF3C8C42A4
:104AC000204601D9002009E00578BD4204F1010427
:104AD000F5D10CEB0405D618A54201D1BDE8F08153
:104AE00015F8018D16F801EDF045F5D0E7E7000067
:104AF000034611F8012B03F8012B002AF9D1704766
:104B00006F72672E6172647570696C6F742E41529A
:104B10004B5F47505300000040A2E4F164689106E7
:104B20000041A3E5F265699207000000426164203C
:104B300043414E496661636520696E6465782E0065
:104B400080000000008000000000800000000000E5
:104B500000000000B1190008F521000851210008EB
:104B6000F1190008FD190008091C0008C119000806
:104B7000D1190008C5190008CD190008C919000885
:104B8000251B0008D519000819250008C9240008AC
:104B9000E5190008F91A000863300000984B000876
:104BA000904A0020A04C002000400000004000007F
:104BB0000040000000400000000001000000020072
:104BC00000000200000002006D61696E0069646C03
:104BD00065000000A000902A00000000AAAAAAAA6E
:104BE00050000024FFFB0000007700000090090047
:104BF0000100000500000000AAAAAAA5010000808B
:104C0000FFCF0000000000000000000000000000D6
:104C100000000000AAAAAAAA00000000FFFF0000EE
:104C20000000000000000000000000000000000084
:104C3000AAAAAAAA00000000FFFF000000000000CE
:104C4000000000000000000000000000AAAAAAAABC
:104C500000000000FFFF0000000000000000000056
:104C60000000000000000000AAAAAAAA000000009C
:104C7000FFFF000000000000000000000000000036
:104C800000000000AAAAAAAA00000000FFFF00007E
:104C90000000000000000000000000000000000014
:104CA0000A000000000000000300000000000000F7
:104CB00000000000000000006D4500085945000894
:104CC00095450008814500088D4500087945000894
:104CD0006545000851450008A14500080000000096
:104CE000510000000000000000000700000000006C
:104CF00040420F00FE2A0100D204000020230020C1
:104D000000000000000000000000000000000000A3
:104D10000000000000000000000000000000000093
:104D20000000000000000000000000000000000083
:104D30000000000000000000000000000000000073
:104D40000000000000000000000000000000000063
:104D50000000000000000000000000000000000053
:00000001FF
